:1000000083128A116528840000308A000408820760
:10001000503400340F34003430343C340034003475
:1000200030343A340034003430343B34003400345B
:100030005034003400340034C0340334A734003466
:10004000C034043402340034C034053499340034EC
:10005000C0340334273400343034083400340034DE
:10006000840000308A0004088207303432340034BF
:100070000034303433340034003430343634003417
:100080000034303437340034003430343834003401
:100090000034303439340034003430343A340034ED
:1000A000003430343B340034003430343F340034D6
:1000B000003430343E340034003430342F340034D3
:1000C000003430342E34003400340C30840080018D
:1000D000840A50300402031C672800308500003079
:1000E00086008316F4308500003086008312831664
:1000F0008030810000308B008312F822F822F82231
:10010000F822F8229A224430D2226130D22274306E
:10011000D2226130D2222030D2227230D2226530F7
:10012000D2226130D2226430D2226930D2226E30A3
:10013000D2226730D2222E30D2222E30D2222E303E
:10014000D2224030CB222030D2222030D222563050
:10015000D2226530D2227230D2227330D22269305C
:10016000D2226F30D2226E30D2222030D2223130D1
:10017000D2222E30D2223030D2223230D22264002B
:1001800083120511853084000011F0220015F4223D
:100190000011F0220015F4229201930191010A301E
:1001A0008F00110896000310960D960D1208160781
:1001B00094000320950000301206031DE42803304C
:1001C0001306031DE428950115083B21EA22920A33
:1001D00004301206031DD1289201F222930A043042
:1001E0001306031DD1289301910A0F081106031D60
:1001F000D1280000F2229201930191010A308F0070
:1002000040309000110896000310960D960D1208CC
:10021000160794003020950000301206031D1529A2
:1002200003301306031D1529950115083B21EA2209
:100230008D0902301302031D262902301202031D0C
:100240002629100884000D088000900A920A0430C4
:100250001206031D02299201F222930A04301306AA
:10026000031D02299301910A0F081106031D02299B
:1002700000005F21FB2864008E008E098D010511AE
:100280008530840000119630042396300423001535
:100290006400083096008E0C03184F295129001570
:1002A000532900115329963004238D0C8D13051901
:1002B0008D1796300423960B4B2900150800B522A4
:1002C000E8222030D2224830C81F6829C801C9015D
:1002D00048300C226D30D2224130D2226830D222F6
:1002E0006D304A2241304A2268304A220D304A227B
:1002F0002030D2224430F6214630F621440846020E
:10030000031C872945084702031C872995292D309E
:10031000D2222D304A220310C50DC40DC50DC40DC7
:10032000C50DC40D44300C22A2292B30D2222B3013
:100330004A220310C70DC60DC70DC60DC70DC60D49
:1003400046300C226D30D2224130D2226D304A220A
:1003500041304A220D304A222030D2222030D2228F
:100360004030CB222030D2224230F62142089F007A
:1003700043089E0003109E0D9F0D0310C30DC20D78
:10038000C30DC20DC30DC20DC30DC20D1E08C302A5
:10039000031C9F0A1F08C20242300C226D30D22279
:1003A0005630D2226D304A2256304A220D304A222F
:1003B0002030D2222030D2222030D2224030F621EA
:1003C0004108003CC100031CC00A4008043CC000B6
:1003D0000310C10DC00DC10DC00D40302C224330A3
:1003E000D22243304A220D304A22080084000008FD
:1003F0009F00840A00089E009D0003109F0D9E0D23
:100400009F0D9E0D1D089F0403309E051F08800050
:1004100084031E0880000800840000089B00840AF2
:1004200000089C0077221E086322A100D222210826
:100430004A221E086622A100D22221084A221F0851
:100440006322A100D22221084A221F086622A100AD
:10045000D22221084A220800840000089B00840A56
:1004600000089C0077221E086322A100D2222108E6
:100470004A221E086622A100D22221084A222E30DA
:10048000D2222E304A221F086322A100D222210844
:100490004A22080064008C0085111D3004230830B6
:1004A00097008C0C031C552A572A8511592A85154B
:1004B000592A1D300423970B512A85151D3004231A
:1004C0001D30042308008400840E682A8400682AF2
:1004D00002308A000F300405820730343134323460
:1004E0003334343435343634373438343934031013
:1004F000103099009D019E019F019C0D9B0D9F0D49
:100500009E0D9D0D990B852A08001F3084008F22B7
:100510001E3084008F221D3084008F227D2A0330FC
:1005200000079A009A198000303000079A009A1B41
:10053000800008008510E422A522A522A522A92278
:10054000AD22B122BE22BA2208003030A000DA2249
:1005500008002030A000DA2208002830A000CF22B6
:1005600008000130A000CF2208000230A000CF22F6
:10057000E82208000630A000CF2208000D30A000BD
:10058000CF22E82208001C30A000CF22080040380B
:10059000A000CF2208008038A000CF2208008510DC
:1005A000E222D62A8514A000E222D62ADA22A00E60
:1005B000DA22080020088600E2220514E222051053
:1005C000E2220800FA30042B0130FA2A0230FA2A1B
:1005D0000530FA2A0930FA2A0A30FA2A0F30FA2AA4
:1005E0001430FA2A2430FA2A2830FA2A3530FA2A26
:1005F000C830FA2A9600D7300423D7300423D730E6
:100600000423960BFB2A080098006400980B052B26
:040610000800092BAA
:02400E00F63F7B
:00000001FF
